:040000008A01372812
:08000800A6000308A7001A0876
:10001000AA0028181428FE302A06031912282A08D4
:10002000EC20322828143228A818282828192D282E
:1000300011302A060319242812302A06031926280B
:100040002A08F42028103228A8143228281532282B
:10005000A81028102A0895003228281128102A08EC
:100060009B00322827088300A60E260E09002B21AC
:100070008501A8018316FC308500FF308600B93069
:1000800087008113831297019101FF309200FF30A6
:1000900095000B1183168C1083128C102C30970056
:1000A000921412159D0185309B002C309D008F20ED
:1000B000AD2083161813181218150C3099009816D5
:1000C000831298019817181683168D018C018C16CF
:1000D00083128C018D018B010B178B17FF300606E5
:1000E00003196E28060899000230A5008230A4008A
:1000F0000A30A300FF30060603198C28A30B7A28C8
:10010000A40B7A28A50B7A28FF30060603198C2841
:100110000608990024218428172117216E281C2104
:100120001C211C211C2103100330FC201C21051460
:100130000510172105140510172103100230FC20AB
:1001400017212830F4200830F4200130F4201C213D
:100150000630F4200F30F420080084010408840ADB
:10016000C92000380319B628EC20AE28C030F4208E
:1001700084010408840ADB2000380319C128EC201C
:10018000B9282B212B212B212B212B210130F420CD
:10019000080082074C3443344434203443346F34F1
:1001A0006E34743472346F346C34203431342E3401
:1001B0003134203400348207283463342934203425
:1001C00041346E34643472346534203444346534DC
:1001D00079346B3420340034A100210E0314FC2048
:1001E00021080314FC200800A100210E0310FC20AC
:1001F00021080310FC200800A200A20E0630A00077
:1002000085148510A00B0029051485148510051090
:10021000850D851485100430A000A20D0510850DF4
:1002200085148510A00B0D29051405100800D83081
:10023000013E031C182908000430A0001830013EBC
:100240000319A00B1F2908000230A5000530A400E7
:10025000B930A30032290230A5008730A4009930BC
:10026000A3003229A30B3229A40B3229A50B322972
:02027000080084
:02400E00713F00
:00000001FF
